:020000040000FA
:020000000528D1
:08000800E82903138316003000
:100010009F00C3308600870108308100813099003D
:100020001812181598160C148C16031383128B16BD
:100030000030A7000030A300A5000330AB0006117C
:10004000871231309000CF308F002B308E008130FE
:100050009F00981718160B17031383163C30920055
:100060008710071187170313831268206D20230858
:10007000950025089B00073092000F3097009D00E7
:100080008612A101A2010530B000B1008B179521A5
:10009000A221FF30C420C321AA20AF212430B520E3
:1000A0005430B5205330B5202D08B5202E08B5208A
:1000B0002F08B5208B132B1C63288712AB1C6528D7
:1000C00006118B17492887165E2806158B174928B5
:1000D0000030970007128711080000309D000710BC
:1000E0008611080022187828221E7D282212221448
:1000F00087110F30970007160800221568200800A6
:10010000A2188628A21E8B28A212A21486110F30D4
:100110009D0007140800A2156D200800221C9428D9
:10012000221E99282212221007120F3097008715DD
:100130000800221568200800A21CA228A21EA728D9
:10014000A212A21007100F309D0086150800A215FC
:100150006D2008000130C4201F151F19AD281E088E
:10016000AD002D0C7F39AD0008000C1EB52899009C
:1001700008000A30FB00FB0BBE28C328B630FC0089
:10018000FC0BC028BB280800FD00FD0AFD0BC92898
:10019000CB28B920C6280800031383168610031342
:1001A000831286108E210313831686140313831281
:1001B0008921013086180030B300892133080800F6
:1001C0000313831606100313831206108E210313E4
:1001D0008316061403138312892101300618003098
:1001E000B300892133080800031383168610031314
:1001F000831286107E21B300331886148921861459
:10020000892133080313831686140313831208000D
:100210000313831606100313831206107E21B30006
:100220003318061489210614892133080313831611
:100230000614031383120800B3000830B200330819
:10024000F420B300B30C33087F390318803EB20B9F
:1002500020290800B3000830B20033080821B30099
:10026000B30C33087F390318803EB20B2E290800E7
:100270000313831686100313831286107E21031343
:100280008316861403138312FE39013E861CFE3941
:10029000B30089218921330808000313831606104F
:1002A0000313831206107E2103138316061403130F
:1002B0008312FE39013E061CFE39B30089218921D3
:1002C00033080800B3000830B20033083821B30007
:1002D000B30C33087F390318803EB20B662908003F
:1002E000B3000830B20033084D21B300B30C33081B
:1002F0007F390318803EB20B74290800000000000B
:1003000000000000000008001930B400B40B86297A
:1003100008006430B500B50B8B2908000930B60021
:10032000B60B9329080089219029CC20CC301C21C0
:100330004E301C2100301C2100301C2100301C21BB
:10034000CC200800E020CC302A214E302A21003079
:100350002A2100302A2100302A21E0200800CC2068
:10036000CC301C2144301C216430C420CC20CC3043
:100370001C21BE301C216221B8006221B700CC20B4
:10038000D721AE000800E020CC302A2144302A21B9
:100390006430C420E020CC302A21BE302A217021D4
:1003A000B8007021B700E020D721AF00080003108B
:1003B000B80CB80CB80CB80C0F30B8050310B70D5A
:1003C000B70DB70DB70DF030B70538083706080080
:1003D000FF000308FE0003138312031383120C189B
:1003E000F6290B19102A8C1A1C2AAB2ACF308F0041
:1003F0002B308E000C10A21D052AB10B042AA21668
:100400000530B100A211052AA212221DAB2AB00BA1
:100410000E2A22160530B0002211AB2A2212AB2A76
:10042000A90303198612AA0B1A2A8616FF30AA00FE
:100430002808A9000B11AB2A1A08A0002118262AA7
:1004400024302002031DAB2A2114AB2AA1182E2A26
:1004500054302002031DAA2AA114AB2A2119362ADE
:1004600043302002031DA92A2115AB2AA1193C2AD9
:100470002008A300A115AB2A211A422A2008A500B2
:100480002116AB2AA11A482A2008A700A116AB2AD8
:100490002008AB000030270203195C2AA71F5F2A3F
:1004A0002708A800A8092808013EA8000310A80CE6
:1004B00028081E3EA800672A1E30A800672A2708C1
:1004C000A8000310A80C1E30AC0028082C02A800BD
:1004D0000030230203197B2AA31F7E2A2308A400CD
:1004E000A4092408013EA4000310A40DA40D2408AF
:1004F00095008E20872A95016820872A2308A4006A
:100500000310A40DA40D240895008800722000306B
:10051000250203199A2AA51F9D2A2508A600A609C7
:100520002608013EA6000310A60DA60D26089B0076
:100530009C20A52A9B016D20A52A2508A600031052
:10054000A60DA60D26089B008020A1122112A11144
:100550002111A11021107E088300FF0E7F0E0900DB
:084000000100090004000900A1
:02400E00323F3F
:00000001FF
